:1000000026C040C027C13EC03DC03CC03BC03AC036
:1000100039C038C037C036C035C034C033C032C034
:1000200031C068656C6C6F2E667464692E34342E32
:100030006563686F2E696E746572727570742E6375
:100040003A20796F7520747970656420000011245E
:100050001FBECFE5D1E0DEBFCDBF10E0A0E6B0E02F
:10006000E0EEF2E002C005900D92A036B107D9F79C
:1000700010E0A0E6B0E001C01D92A436B107E1F7A0
:1000800022D12CC1BDCFDC01FA0110828C918623D4
:10009000E9F78CE18A95F1F788E38A95F1F78C917D
:1000A000862319F081E0808301C0108288E38A955D
:1000B000F1F78C91862319F080818260808388E338
:1000C0008A95F1F78C91862319F080818460808372
:1000D00088E38A95F1F78C91862319F080818860F6
:1000E000808388E38A95F1F78C91862319F08081CB
:1000F0008061808388E38A95F1F78C91862319F0DB
:1001000080818062808388E38A95F1F78C918623D1
:1001100019F080818064808388E38A95F1F78C915F
:10012000862319F080818068808388E38A95F1F7BF
:100130008CE18A95F1F70895FC018081962F9095C6
:100140008923808388E38A95F1F7242F332727FDBD
:10015000309520FF03C08081862B02C080818923D7
:10016000808388E38A95F1F721FF03C08081862B85
:1001700002C080818923808388E38A95F1F722FF7A
:1001800003C08081862B02C080818923808388E31D
:100190008A95F1F723FF03C08081862B02C08081FE
:1001A0008923808388E38A95F1F724FF03C0808147
:1001B000862B02C080818923808388E38A95F1F7AA
:1001C00025FF03C08081862B02C080818923808324
:1001D00088E38A95F1F726FF03C08081862B02C051
:1001E00080818923808388E38A95F1F747FF04C0E3
:1001F0008081862B808303C080819823908398E33D
:10020000892F8A95F1F78081862B80839A95F1F763
:100210000895EF92FF921F93CF93DF93EA01EE24AC
:10022000FF24FE0114918BE390E062E0412F84DF14
:100230000894E11CF11C2196112399F71092630098
:10024000F0926200E0926100DF91CF911F91FF90E8
:10025000EF9008951F920F920FB60F9211242F93D3
:100260003F934F935F936F937F938F939F93AF933E
:10027000BF93EF93FF9389E390E061E040E650E0A5
:1002800002DF8BE390E062E042E250E0C2DF8BE30A
:1002900090E062E0409160004FDF8BE390E062E02D
:1002A0004AE04ADFFF91EF91BF91AF919F918F910B
:1002B0007F916F915F914F913F912F910F900FBE62
:1002C0000F901F90189580E886BD16BCD99AD19AD8
:1002D0008BB780618BBF909A7894FFCFF894FFCF53
:00000001FF
